:100000000C94C7010C94FF010C94FF010C94FF01A8
:100010000C94FF010C94FF010C94FF010C94FF0160
:100020000C94FF010C94FF010C947E1D0C94501E47
:100030000C94BD170C94FF010C94FF010C94FF016C
:100040000C94FF010C94FF010C94FF010C94FF0130
:100050000C94FF010C9445180C94FF010C94FF01C3
:100060000C94FF010C94FF010C94FF010C94FF0110
:100070000C94FF010C94FF010C94FF010C94FF0100
:100080000C94FF010C94FF010C94FF010C94FF01F0
:100090000C94FF010C94FF010C94FF010C94FF01E0
:1000A0000C94FF010C94FF010C94FF01B705B705F8
:1000B000E305E3054B067607760776076906020730
:1000C00013071307BD1EE41EDC1FE41EDC1F301FD8
:1000D000531FDC1FAA1FB91F2B0014001A000800B1
:1000E000150017001C0018000C00120013002A0055
:1000F000E00004001600070009000A000B000D00D4
:100100000E000F0033003400E1001D001B0006004C
:100110001900050011001000360037003800E50016
:10012000E000E200E30028000000000000002C00D6
:10013000E60029000000E40044454255473A2064A7
:10014000697361626C65642E0A0044454255473A02
:1001500020656E61626C65642E0A000A00253032EB
:1001600058006C65645F7461736B3A20004F6E6574
:1001700073686F743A206163746976653A20256408
:100180000A000A002530313662003A20002530325C
:1001900058000A722F632030313233343536373805
:1001A000394142434445460A000A0025303258206E
:1001B000006B6579626F6172645F7265706F7274F3
:1001C0003A200064656C5F6B65795F6269743A2000
:1001D00063616E27742064656C3A20253032580ABA
:1001E000006164645F6B65795F6269743A20636182
:1001F0006E2774206164643A20253032580A005B0F
:10020000735D005B575D005B535D005B525D005B9F
:10021000445D005B435D00100343006100720061B8
:1002200000760061006E0000002203540068006543
:1002300000560061006E0020004B006500790062EE
:10024000006F006100720064007300000004030985
:100250000409025B00030100A0FA09040000010385
:10026000010100092111010001224000070581035D
:100270000800010904010001030000000921110127
:100280000001226D0007058203200001090402001D
:1002900002030000000921110100012222000705CC
:1002A000830320000107050303200001120100025F
:1002B00000000008AEFE4488010001020001063182
:1002C000FF0974A1010975150026FF009520750826
:1002D00081020976150026FF00952075089102C05D
:1002E00005010980A101850319012AB7001501261E
:1002F000B700950175108100C0050C0901A10185A9
:100300000419012AA002150126A002950175108189
:1003100000C005010906A1018506050719E029E7C6
:10032000150025019508750181020507190029EFBF
:100330001500250195F075018102050819012905AF
:10034000950575019102950175039101C00501099B
:1003500006A101050719E029E71500250195087593
:100360000181029501750881010507190029FF1512
:100370000026FF009506750881000508190129056A
:10038000950575019102950175039101C000112435
:100390001FBECFEFDAE0DEBFCDBF04B603FE18C04C
:1003A0008091A3029091A402A091A502B091A6020F
:1003B0008730904BA740B04B59F41092A302109293
:1003C000A4021092A5021092A602E0E0F8E30995BB
:1003D00011E0A0E0B1E0E4EEF0E402C005900D927F
:1003E000A239B107D9F722E0A2E9B1E001C01D921C
:1003F000A33AB207E1F70E94C0130C9470200C944A
:100400000000FF93EF93E0919201F09193013097F8
:1004100009F00995EF91FF910895FC0185918030D5
:1004200011F0EFDFFBCF0895FF27E0E230E247FF56
:100430000CC0419597FF09C0EDE2609570958095DD
:100440009095611D711D811D911D27FF02C0219591
:1004500030E350E2AA27660F771F881F991FAA1F53
:10046000A41710F0A41B63955A95A9F7AA3008F0B9
:10047000A95FA05DAF93F3956115710581059105A5
:1004800041F7ED3211F4EF93F395F21718F43F931F
:10049000F395FBCF8F91B5DFFA95E1F70895E991D8
:1004A000F9918591803021F0853219F0AADFF9CFDA
:1004B000089520E0E89455915532C1F3503311F47A
:1004C000689455915A3348F4505390F3220F022EFA
:1004D000220F220F200D250FF4CF0EF421958991C4
:1004E0009991533619F3533729F1533559F1BC011A
:1004F00088279927E8945C3621F48991999168942A
:100500005591543639F446EF7EF077FF0DC08FEFEA
:100510009FEF0AC055374AE039F0583540E121F0E5
:10052000523642E009F00895FF93EF937DDFEF919B
:10053000FF91B7CFFF93EF93FC0181918030B9F326
:1005400060DFFBCFFF93EF9368DFF1CFDF93CF93B3
:10055000CDB7DEB72596A3DFCF91DF91089581E077
:10056000089581E008950C94B10208950C94B502A9
:100570001F93CF93DF9300D000D01F92CDB7DEB78B
:1005800049835A836B833091950189819A81311116
:1005900014C0662359F0222349F00E94AF09182F96
:1005A000682F89819A810E94580903C00E9483099B
:1005B000182F69817A81812F04C00E94AF09698157
:1005C0007A810F900F900F900F900F90DF91CF9145
:1005D0001F910C94E710FC01262F4081518162810C
:1005E000738184810C94B80281E00895CF93DF93E6
:1005F000EC0160E00E94EB02BE01DF91CF910C9410
:10060000B6020C9471120C946D1208950E940208A7
:100610000E9405032FEF84E39CE02150804090402E
:10062000E1F700C000000C946B180F931F93CF9359
:10063000DF938C0161E00E94EB02EC01B8010E94A3
:10064000B302882309F45BC0B801CE010E94B9153A
:10065000882309F454C0B801CE010E94CD13882329
:1006600009F44DC0B801CE010E941515882309F484
:1006700046C0F80182818823D9F1CF3D8CE5D807A7
:1006800079F140F4C115FCE5DF0791F0C130DC459C
:1006900091F02EC0CC35EDE5DE0741F1CD35FDE51D
:1006A000DF0709F1CB35DD4519F50E94460E20C064
:1006B0000E94060324C080914802C82FC095C170D3
:1006C000C0FB80F980934802CC2329F08AE491E0B2
:1006D0000E940D0214C088E391E00E940D0210C038
:1006E0000E94FA0E0CC00E943D0E02C00E94490EEC
:1006F000C801DF91CF911F910F910C94AF02C0E020
:100700008C2FDF91CF911F910F9108950E949F1719
:100710000C94C4030E94C7030C94A5178295982FCC
:10072000937344E0949F900111248C7C8695869568
:10073000282B822F8575880F2A7A2695822B08957B
:10074000CF93DF93D92F0E948E03C82F8D2F0E9445
:100750008E032C2F30E0322F2227A901482BCA010B
:10076000DF91CF91089508950C94B30381E008952B
:100770000C94B6030895CF93C82F0E94B4038C2F16
:100780000E94B803CF91089580E00C94BB030E94AF
:1007900015160C94BB03CF930E941516C82F809199
:1007A0009401C81741F1C09394018091480282FFDF
:1007B0001EC080FF04C082E691E00E940D0280917D
:1007C000480280FF0CC01F92CF938DE591E09F936C
:1007D0008F930E94A6020F900F900F900F90809120
:1007E000480280FF04C08BE591E00E940D028C2F2F
:1007F000CF910C94BB03CF910895CF93DF93CDB7E6
:10080000DEB72B970FB6F894DEBF0FBECDBF4F8378
:10081000588769877A878B8761110E94750D9E01C1
:100820002F5F3F4F86E0F90111928A95E9F785E045
:10083000FE013796D90101900D928A95E1F78981E1
:100840009A814C815D81452B31F09F3F31F491E0DD
:100850008F3F19F403C091E001C090E090FF09C000
:1008600049815A816B817C818D819E810E94960C89
:1008700005C0C9010E94F4028111F2CF2B960FB678
:10088000F894DEBF0FBECDBFDF91CF910895FC017C
:10089000808191810E94F1090895CF93882309F402
:1008A0009CC0C82F8238C1F40E94151681FD95C0E6
:1008B00069E380910201909103010E945A170E94FE
:1008C000970D2FEF81EE94E0215080409040E1F7AA
:1008D00000C0000069E319C0833801F50E941516B5
:1008E00080FD7BC063E580910201909103010E942D
:1008F0005A170E94970D2FEF81EE94E0215080400F
:100900009040E1F700C0000063E580910201909102
:1009100003010E946517CF910C94970D8438C1F4A0
:100920000E94151682FD59C067E4809102019091E2
:1009300003010E945A170E94970D2FEF81EE94E059
:10094000215080409040E1F700C0000067E4DDCF17
:100950008CEF8C0F813AD0F46C2F80910201909132
:1009600003010E94B816882349F06C2F8091020180
:10097000909103010E9465170E94970D6C2F809142
:100980000201909103010E945A17C5CF80E28C0F9B
:10099000883048F4C77081E001C0880FCA95EAF733
:1009A0000E94580DB8CFEBE5EC0FE33040F4F0E0D7
:1009B000E15CFE4F808190E0CF910C947616C85A8E
:1009C000C73158F4EC2FF0E0EE0FFF1FEF5EFE4F43
:1009D00080819181CF910C948C16CF9108958823BA
:1009E00009F45BC0682F823879F40E94151681FFE4
:1009F00054C069E380910201909103010E945A174B
:100A00000E94970D69E310C08338B1F40E94151657
:100A100080FF43C063E580910201909103010E9431
:100A20005A170E94970D63E580910201909103018E
:100A30000E9465170C94970D843879F40E9415165E
:100A400082FF2BC067E480910201909103010E9414
:100A50005A170E94970D67E4E7CF8CEF860F813A13
:100A600018F380E2860F883048F4677081E001C097
:100A7000880F6A95EAF70E945E0DDCCF8BE5860F42
:100A8000833020F480E090E00C947616685A673149
:100A900020F480E090E00C948C1608951F93CF937F
:100AA000DF93182FEB010E944D04209741F08FE94E
:100AB0009FE00197F1F700C000002197F6CF812F4A
:100AC000DF91CF911F910C94EF04893319F060E00E
:100AD00070E002C060E570E00C944E05882321F0C0
:100AE0000E94580D0C94970D0895882321F00E94C0
:100AF0005E0D0C94970D0895CF92DF92EF92FF92C6
:100B00000F931F93CF93DF937C01D62FC72FFC0148
:100B10001281058102950F700E944E0D8823B9F055
:100B20001123A9F08C2F807F803421F080E28D0F7B
:100B3000883068F08091810282FD09C082E00E94C5
:100B4000F70D0E944E0D91E0D82ED92601C0D12C70
:100B5000CC2EC2948FE0C8228C2D90E08C30910571
:100B600008F0C4C1FC01EA5AFF4F0C941B208C2FE3
:100B7000807FCF70882311F0C295C07F112399F038
:100B8000CC2309F49FC180E28D0F883010F0D11181
:100B900004C08C2F0E94580D03C08C2F0E94680D3A
:100BA0000E94970D8FC18D2F0E94EF04CC2309F472
:100BB0009DC180E28D0F883038F1DD2329F18C2F23
:100BC0000E946E0D24C08C2F807FCF70803211F078
:100BD000C295C07FDD2319F0D130A1F13DC08091D5
:100BE000810282FF17C0112349F0CC2329F08C2FFA
:100BF0000E94580D0E94970D80E065C180E00E9420
:100C0000EF04CC2309F472C18C2F0E945E0D0E9468
:100C1000970D6CC1112371F0002341F0013031F4C4
:100C20000E94780D8C2B0E94800D60C10E94780D6F
:100C30008C2B1DC0002319F0013009F457C10E940C
:100C40008D0D25C0112321F0063008F04FC10EC0D4
:100C5000053008F04BC11BC0112361F0002331F0B7
:100C6000F701858180FF2EC18F7085838C2F0E94B4
:100C70006E053CC1002359F0D93309F034C1FFEFB0
:100C800007EE13E0F15000401040E1F72AC18C2F2D
:100C90000E9475052BC18C2F86958695837019F05F
:100CA000813061F023C1112321F08D2F9C2F93708F
:100CB00002C080E090E00E94761620C1112321F04E
:100CC0008D2F9C2F937002C080E090E00E948C16C4
:100CD00015C18C2F837009F047C011110BC12D2F46
:100CE000229526952770220F220F6D2F6F70862F69
:100CF00090E0A0E0B0E0022E04C0880F991FAA1F68
:100D0000BB1F0A94D2F7D4FF10C04FE050E060E060
:100D100070E004C0440F551F661F771F2A95D2F755
:100D2000409550956095709503C040E050E0BA0141
:100D3000C695C695C3708A019B01082B192B2A2BD7
:100D40003B2BC901B801C23049F058F4C13019F049
:100D50000E946E08CFC00E945C08CCC00E94800830
:100D6000C9C00E945A08C6C0112319F08C2F817087
:100D700001C08695882309F4BDC02D2F22952695A4
:100D80002770220F220F6D2F6F70862F90E0A0E04A
:100D9000B0E0022E04C0880F991FAA1FBB1F0A943F
:100DA000D2F7D4FF10C04FE050E060E070E004C024
:100DB000440F551F661F771F2A95D2F7409550950F
:100DC0006095709503C040E050E0BA01C695C695A5
:100DD000C3708A019B01082B192B2A2B3B2BC901BD
:100DE000B801C23049F058F4C13019F00E943309FB
:100DF00081C00E9421097EC00E9445097BC00E94DB
:100E0000940878C0CF70112339F08C2F0E94BA0853
:100E10008D2F0E946E056EC08D2F0E9475058C2F40
:100E20000E94DB0867C0D23F21F128F4D03F41F097
:100E3000D13FC1F043C0D33F19F1D43F79F03EC058
:100E4000112341F0053008F051C08C2F8F710E94A2
:100E500000094CC0063008F049C0F7CF80918102EC
:100E600082FF18C0112339F08C2F8F710E94BA08AD
:100E70003DC01123C9F38C2F8F710E94DB0836C04F
:100E8000112329F08C2F8F710E94A5082FC00E947A
:100E9000A0082CC0112349F0CF718C2F0E94BA08F2
:100EA00063E08C2F0E94DC0D21C081E00E94F70DD1
:100EB0000230E0F082E00E94F70D18C0112331F0FB
:100EC000002391F28D2F0E944D0410C0002399F24F
:100ED000D93349F41FEF27EE33E011502040304062
:100EE000E1F700C000008D2F0E94EF0488EF8C0D09
:100EF000843020F40E9415160E94BB03DD20C9F047
:100F00000E944A0D80FD15C0F70112820E94440D17
:100F10000E94BA08C7010E94BA070E94440DDF91DF
:100F2000CF911F910F91FF90EF90DF90CF900C9495
:100F3000DB08DF91CF911F910F91FF90EF90DF9031
:100F4000CF9008950F931F93CF93DF93EC016881A7
:100F500079818A810E94FC098C010E9457090E94B4
:100F60004808B801CE010E947C05DF91CF911F9106
:100F70000F910895CF93DF93EC01988189812B81A4
:100F80003C81232B31F08F3F31F481E09F3F19F4F6
:100F900003C081E001C080E080FD1DC0CE010E9441
:100FA0001503811110C00E944E0D8823A1F08A8183
:100FB000882389F08091810282FD0DC082E0DF915B
:100FC000CF910C94F70DCE010E94A207CE01DF91C4
:100FD000CF910C94F602DF91CF91089580E090E0DC
:100FE0000E94761680E090E00E948C160E94750D9B
:100FF0000C94970D80910201909103010E9470174B
:101000000C94EE070E94650D0C94FA0792959F7060
:10101000963079F010F4925001C09A50923068F4F2
:10102000803F69F018F4883E40F409C0843F29F4F9
:1010300006C0883E20F0813F11F080E0089581E0F5
:101040000895FC01808191810E94F1090E940608A7
:101050000895CF93DF9300D000D01F92CDB7DEB7B5
:101060000F900F900F900F900F90DF91CF910895F8
:10107000CF93DF9300D000D000D0CDB7DEB7269657
:101080000FB6F894DEBF0FBECDBFDF91CF910895AC
:10109000089508950C9449080C944A080E944C083D
:1010A0006093B8017093B9018093BA019093BB012A
:1010B0000C94EE070C944E080F931F930091B80107
:1010C0001091B9012091BA013091BB01602B712BB5
:1010D000822B932B1F910F910C944E080F931F930B
:1010E0000091B8011091B9012091BA013091BB0172
:1010F00060237123822393231F910F910C944E0838
:101100000F931F930091B8011091B9012091BA017A
:101110003091BB0160277127822793271F910F9180
:101120000C944E080C9449080E9492086093B401F4
:101130007093B5018093B6019093B7010C94EE07BC
:1011400060E070E0CB010C9494080F931F9341E092
:1011500050E060E070E08A019B0104C0000F111FA5
:10116000221F331F8A95D2F7C901B8011F910F9131
:101170000C9494080F931F9341E050E060E070E0FE
:1011800004C0440F551F661F771F8A95D2F78091C0
:10119000B4019091B501A091B601B091B7018A0157
:1011A0009B01082B192B2A2B3B2BC901B8011F913E
:1011B0000F910C9494080F931F9341E050E060E06E
:1011C00070E004C0440F551F661F771F8A95D2F741
:1011D00040955095609570958091B4019091B501BE
:1011E000A091B601B091B7018A019B010823192390
:1011F0002A233B23C901B8011F910F910C94940835
:101200000F931F9341E050E060E070E004C0440F92
:10121000551F661F771F8A95D2F78091B401909170
:10122000B501A091B601B091B7018A019B010827D1
:1012300019272A273B27C901B8011F910F910C9448
:1012400094080F931F930091B4011091B501209160
:10125000B6013091B701602B712B822B932B1F911C
:101260000F910C9494080F931F930091B401109167
:10127000B5012091B6013091B7016023712382231B
:1012800093231F910F910C9494080F931F93009137
:10129000B4011091B5012091B6013091B7016027DA
:1012A0007127822793271F910F910C94940808951A
:1012B0002CE0929F800D1124E82FE695E695E695A7
:1012C000877051E001C0550F8A95EAF785E0E89FE5
:1012D000F0011124EA56FE4F20E030E070E040813A
:1012E000CB01022E02C0969587950A94E2F7817091
:1012F000819584278523842781932F5F3F4F253055
:10130000310569F708952CE0929F800D1124682F14
:10131000669566956695982F977085E0689FB001F1
:10132000112440E050E080E0FB01E40FF51FEA5695
:10133000FE4F208130E0092E02C0369527950A9491
:10134000E2F721703327042E01C0220F0A94EAF736
:10135000822B4F5F5F4F4530510531F70895BF92A3
:10136000CF92DF92EF92FF920F931F93CF93DF9371
:101370008C01C090B401D090B501E090B601F0901E
:10138000B7018091B8019091B901A091BA01B091D3
:10139000BB01C82AD92AEA2AFB2ACFE1D0E0D7012B
:1013A000C6010C2E04C0B695A795979587950A940B
:1013B000D2F780FD04C0219790F7B12C07C0BC2E56
:1013C000B8018C2F0E94FA100197A9F38B2DDF91A1
:1013D000CF911F910F91FF90EF90DF90CF90BF9032
:1013E0000895CF93DF93EC010E94AF09BE010E94E4
:1013F000FA10DF91CF9108951F93CF93DF93EB0104
:1014000090919501992321F0CB010E94F10913C01D
:10141000882349F0CB010E94AF09182F682FCE0115
:101420000E94580904C0CB010E948309182FBE01F5
:10143000812F0E94FA10DF91CF911F9108951F9381
:10144000CF93DF93C091BC0116E08091BD01C81716
:1014500099F0D0E01C9FF0011D9FF00D1124E25483
:10146000FE4F4081518162817381848195810E9408
:1014700038082196C770E9CFDF91CF911F91089569
:101480004091EE015091EF016091F0017091F101F6
:101490008091F2019091F3010C943808EF92FF9241
:1014A0000F931F93CF93DF938091F30182958F70F9
:1014B00009F065C08091F001882309F460C0809133
:1014C000BC01F090BD011091EE010091EF0160911F
:1014D000F1017091F20191E01F3F09F090E0C0919D
:1014E0000001D0910101292F96E0E92E8F1509F412
:1014F00046C06115710521F00F3F21F030E003C0B7
:1015000031E001C0322F90E030FD36C0E89EF0019E
:10151000E99EF00D1124DF01A254BE4F11963C91BB
:101520001197301329C03C91311326C012963C917B
:101530001297311121C013964D915C911497461B5F
:10154000570B4C175D07C0F48091F3018F708061D9
:101550008093F301ED53FE4F80818F708061808313
:101560008EEE91E00E94BA07DF91CF911F910F910B
:10157000FF90EF900C941F0A01968770B7CFDF9110
:10158000CF911F910F91FF90EF9008959F92AF928E
:10159000BF92CF92DF92EF92FF920F931F93CF9360
:1015A000DF93CDB7DEB761970FB6F894DEBF0FBEFD
:1015B000CDBF8C0185E0F801DE011D9601900D92F2
:1015C0008A95E1F7D8011296EC909091EE01E091A6
:1015D000EF012091F1013091F2012115310531F037
:1015E000EF3F31F481E09F3F19F403C081E001C077
:1015F00080E0B82FB1709B2E80FD47C1D8014C917F
:1016000011965C9111971396AD90BC9014978EEE45
:10161000C82E81E0D82EF090F001B501621B730B4B
:101620002091000130910101FF2009F4D9C080917F
:10163000F3016217730708F095C0282F207F09F087
:1016400052C05E1313C0491311C0FE2CE1100EC02E
:101650008F7080618093F3010E94400AC6010E944E
:10166000BA078091F301F80185834DC1AB2831F0B1
:101670005F3F31F481E04F3F19F403C081E001C0C6
:1016800080E080FD03C081E08E2502C080E090E014
:10169000F82FF170FF2E80FF1CC08091BC012091BB
:1016A000BD0136E0821709F40BC190E0389FF001CC
:1016B000399FF00D1124E254FE4F6181561306C08C
:1016C0006081461303C06281E61203C001968770F1
:1016D000E9CFFE2CEE2009F416C18091F301816060
:1016E0008093F30154C05E1306C0491304C0E11097
:1016F00002C0F80199C0C8010E942108882361F145
:10170000EE2051F12091F301822F82958F7090E0AD
:10171000029774F08091EE019091EF0198878F838A
:101720001986BB86AA862C87CE0107960E94BA0727
:1017300086E0F801AEEEB1E001900D928A95E1F7F6
:101740000E944E0A0E94400A0AC05E1711F1C801A9
:101750000E94210881112CC0C8010E94BA07FF24F1
:10176000F394D1C0282F207F81F77A2DB98AA88AD7
:101770006E2D89890E9429088EEE91E00E94BA0799
:1017800086E0D6011D928A95E9F70E94400AF12C65
:10179000BAC04913DCCFE110DACFF8018583C80164
:1017A0000E94BA0786E0D6011D928A95E9F7ABC080
:1017B000EE2091F22091F301822F82958F7090E0BC
:1017C00002970CF4B5CF8091EE019091EF019A83CE
:1017D00089831B82BD82AC822E83CE010196A6CF67
:1017E0006217730708F044C0FE2CEE2009F4B4CF52
:1017F0005E1330C049132EC02091F30120FD21C09B
:10180000822F82958F70482F50E041155105C9F005
:10181000F80125834F30510541F08F5F982F929545
:10182000907F822F8F70892B8583C8010E94BA0711
:1018300086E0F801AEEEB1E001900D928A95E1F7F5
:101840003CC086E0F801AEEEB1E001900D928A95C1
:10185000E1F759C0C8010E942108811169CF809128
:10186000F30181608093F301C8010E94BA074BC065
:101870007A2DB98AA88A6E2D89890E94290886E066
:10188000D6011D928A95E9F718C0EE2009F464CFBD
:10189000C8010E942108F82E882309F45DCF86E054
:1018A000F801AEEEB1E001900D928A95E1F78EEE6F
:1018B00091E00E9447040E944E0A0E94400A23C001
:1018C0004D875E878D859E850E94F109292F22957F
:1018D0002F70223028F49F7039F0811105C00BC0A1
:1018E000243028F49F7049F4805E883020F0C801CD
:1018F0000E94BA079F2CF92C06C0D80115969C911E
:10190000907F91F7F8CF8F2D61960FB6F894DEBFD8
:101910000FBECDBFDF91CF911F910F91FF90EF9040
:10192000DF90CF90BF90AF909F9008951F93CF937B
:10193000DF93CDB7DEB72C970FB6F894DEBF0FBE9E
:10194000CDBF4F83588769877A878B879C87CE0165
:1019500007960E94C60A8823D1F09F8188852A8530
:101960003B85232B31F08F3F31F481E09F3F19F409
:1019700003C081E001C080E080FD47C04F815885F1
:1019800069857A858B859C850E9438083EC086E0F3
:10199000FE013796DE01119601900D928A95E1F7CE
:1019A000FF81E8856A857B856115710531F0EF3F20
:1019B00031F481E0FF3F19F403C081E001C080E011
:1019C00080FD23C02091BD0130E0C90101968770E0
:1019D00099274091BC0150E084179507F1F1F983F4
:1019E000EA837D836C8396E0929FD001939FB00D34
:1019F0001124A254BE4FFE01319601900D929A958A
:101A0000E1F78093BD010E941F0A16E08091BC019E
:101A10009091BD01891771F1189FC0011124825462
:101A20009E4F0E94C60A882329F1E091BC011E9FA7
:101A3000F0011124E254FE4F408151816281738193
:101A4000848195810E9438088091BC0190E00196C4
:101A5000877099278093BC01D9CF0E940208109209
:101A6000BD011092BC01EEEEF1E086E0DF011D92B7
:101A70008A95E9F72C960FB6F894DEBF0FBECDBF5E
:101A8000DF91CF911F9108958091140285958595DE
:101A9000859508958091140287700895909114029D
:101AA000977081E009F480E00895809137020895ED
:101AB00090913702892B80933702089580959091F9
:101AC00037028923809337020895109237020895D0
:101AD00090913602892B80933602089580959091DB
:101AE00036028923809336020895109236020895B3
:101AF00080911502089508950C947B0D0C947C0D33
:101B00009091810292FD08C090911502981721F0E2
:101B1000809315020C947E0D089580911502882300
:101B200029F01092150280E00C947E0D0895CF9359
:101B3000DF93E0910201F0910301809137028083ED
:101B4000E0910201F0910301908180913602892B8E
:101B5000808380911502882381F0E0910201F09149
:101B600003019081892B8083809102019091030170
:101B70000E94A21681110E948D0DC0910201D09188
:101B8000030140E250E064EF71E0CE010E942120A9
:101B9000892B69F080E2FE01A4EFB1E001900D9283
:101BA0008A95E1F7CE01DF91CF910C942116DF9158
:101BB000CF9108950C947B0D9091810292FD10C0FD
:101BC00098E0899F90011124262B209314020E94F3
:101BD000BA08809114028595859585950C94DA0D47
:101BE0000C94BA081092140280E00C94DA0D209143
:101BF00014028095822380931402982F977099F491
:101C000030E0482F082E000C550B2417350759F0EB
:101C10009091810292FD07C08595859585950E94DA
:101C2000DB080C94F20D0895CF939091810292FB02
:101C3000222720F92817F9F0C82F892FC0FB82F935
:101C40008093810280918002909181020E94760EA1
:101C500082E00E94F70D8091480280FF0CC01F9225
:101C6000CF938DE691E09F938F930E94A6020F90F1
:101C70000F900F900F90CF9108958091810282FB79
:101C8000882780F991E089270C94140E81E00C9448
:101C9000140E80E00C94140E6FEF7FEF80E090E064
:101CA0000C945A2080E090E00E94362021E0893E8A
:101CB0009E4F09F020E0822F089582E090E00C947E
:101CC0002E2083E090E00C942E20CF9384E090E0CF
:101CD0000E942E20C82F82E290E00E942E202C2FFE
:101CE00030E0A901582BCA01CF910895CF93C92F95
:101CF000682F84E090E00E943C206C2F82E290E00C
:101D0000CF910C943C20AB01BC018FE090E00C948F
:101D10004E20AB01BC0183E190E00C944E2060E0CA
:101D200070E0CB010C94890E60E070E0CB010E9462
:101D3000830E0C948F0E69EE7EEF80E090E00E949F
:101D40005A2060E082E090E00E943C2060E083E066
:101D500090E00E943C201092B8011092B9011092BC
:101D6000BA011092BB0160E084E090E00E943C2048
:101D700060E082E290E00E943C2060E085E090E03C
:101D80000E943C2060E086E090E00E943C206FEFE3
:101D900087E090E00E943C2040E050E0BA0188E0FB
:101DA00090E00E944E2060E08DE090E00E943C2098
:101DB00040E050E0BA0188E190E00E944E2060E0EF
:101DC00087E190E00E943C2040E050E0BA018CE1C5
:101DD00090E00E944E2060E070E080E290E00E947F
:101DE0005A2040E050E0BA0188E190E00E944E2085
:101DF0000C94940E0C949B0E682F8EE090E00C9443
:101E00003C200E942A1860934402709345028093FC
:101E10004602909347026093400270934102809380
:101E2000420290934302089585B7806885BF85B7C5
:101E3000806885BF089581E008950C941B0F089574
:101E40000C941F0F0C941F0F0C94220F0C941F0F57
:101E50000C94260F0C941F0F0E94140F89E59AE131
:101E60000E940B160E942A0F0C94280F0E94200F2C
:101E70000C941F0F0E94EE110C94BA030E941518C7
:101E80000E9419130E943A0F0C94240F5F926F92D4
:101E90007F928F929F92AF92BF92CF92DF92EF92FA
:101EA000FF920F931F93CF93DF93CDB7DEB72A979F
:101EB0000FB6F894DEBF0FBECDBF0E942E13C82E02
:101EC00081110E94010F38E3832E32E0932E00E04F
:101ED00010E0502E802F0E9412125C01F4016190DC
:101EE00071904F016826792661147104B1F40F5F77
:101EF0001F4F0430110569F78FEF89838A831B8296
:101F00000E941E188160782F9D838C8349815A819D
:101F10006B818D810E94FD033AC08091480281FD52
:101F20000E941B12D12CEE24E394F12CC3018E21CC
:101F30009F21892B29F10E941D0F8823A9F0DE82A1
:101F40005F82AE20BF2081E0AB2809F480E0888763
:101F50000E941E188160782F9A8789874E815F8141
:101F600068858A850E94FD03000F111FF801E85C57
:101F7000FD4F80819181E826F926F182E08207C039
:101F8000D394EE0CFF1CFCE0DF12D0CFB0CF81E089
:101F9000C11001C080E02A960FB6F894DEBF0FBED4
:101FA000CDBFDF91CF911F910F91FF90EF90DF9008
:101FB000CF90BF90AF909F908F907F906F905F90E9
:101FC00008950E94460F0C94CB03CF93DF930E9499
:101FD000FF10EC01811522E59207E8F5811531E546
:101FE000930708F0B6C0883E910528F5803E91051C
:101FF00008F0E9C0883A910570F4853A910508F037
:102000007AC08130910509F473C008F4D9C00497EF
:1020100008F0D9C0D5C08F3B910508F0D1C0C85A8F
:10202000D0E0CC0FDD1FCE5BDE4F0990D881C02DF4
:10203000CE019464C9C0811540E5940708F069C0D9
:10204000811550E4950708F060C09A9581159F416D
:1020500008F4B9C0B5C0811536E5930728F5811598
:1020600045E5940708F092C0811554E5950708F0FE
:1020700087C0AC0143705527282F26952695C1159A
:10208000D34508F06CC081E090E002C0880F991F32
:102090004A95E2F740E2249F90011124EC01C22B03
:1020A000D32BCE019C6890C081152AE5920780F45D
:1020B000811539E5930708F072C0811548E594074A
:1020C00008F47EC0D82FCC27CE01806F906A7CC0E8
:1020D00090568115904208F073C08D2F8F710E9429
:1020E0009311DD27D0628F71AE01582BCA016CC0ED
:1020F00081E090E069C0C55AD0E0C059DE4F8881C8
:10210000C82FD0E0CE0190645FC0DF70CE01906A2E
:102110005BC074E0969587957A95E1F7282F237038
:102120003C2F337081E090E002C0880F991F3A95F0
:10213000E2F79C68AC01522B9A019C2F9F709695F8
:10214000969550E2959FE0011124C9018C2B9D2B9F
:102150003BC0D82FCC27CE01816F906A35C081E07B
:1021600090E002C0880F991F4A95E2F750E2259F40
:1021700090011124EC01C22BD32BCE019A6824C00C
:10218000D82FCC27CE01846F906A1EC00E94931175
:102190008F7190E0D82FCC27CE01906215C08F7040
:1021A0000E94931194E0D695C7959A95E1F7CF7068
:1021B000D0E0DC2FCC27D0699E01282BC90104C0B8
:1021C00080E090E001C0CE01DF91CF91089520E33F
:1021D000829FC0011124FC012CE0729FE00DF11DD3
:1021E0001124E60FF11DEE0FFF1FE852FF4F8591FE
:1021F000949108950E94E7100E94E50F0895823897
:10220000910569F1B0F48133910509F46DC048F48A
:102210008932910509F463C08A32910509F469C0D5
:1022200008958533910509F455C089339105B9F0B6
:102230000895833E910569F138F4803E9105B1F02F
:10224000823E910509F10895863E9105A9F1873EE8
:102250009105B9F1843E910509F064C023C0209135
:10226000800220FD4FC021FD4DC008958091800265
:1022700080FD44C08091810280FF44C08091800233
:1022800084FD42C083EE4DC08091800282FF38C041
:10229000F5CF8091800282FD33C08091810280FD64
:1022A00031C0ECCF8091810281FF32C080918002E9
:1022B00084FD2AC087EE35C08091800283FF26C04E
:1022C000F5CF8091800283FD21C08091810281FD44
:1022D0001FC0ECCF8091800285FD1CC01DC0809185
:1022E000800285FD19C016C08091800286FD16C04F
:1022F00017C08091800286FD13C010C089E311C011
:1023000082EE0FC080EE0DC080E00BC086EE09C0EB
:1023100084EE07C089E205C085E303C08AE201C0FC
:1023200081E390E008959091800292FF0DC0282FE4
:102330002871283019F4877F846006C0282F247103
:10234000243011F48B7F886093FF0DC0282F2871F3
:10235000283119F4877E846106C0282F2471243126
:1023600011F48B7E88612091810220FF0DC0382FEF
:102370003871383019F4877F816006C0382F317189
:10238000313011F48E7F886021FF0DC0282F287115
:10239000283119F4877E816106C0282F21712131EF
:1023A00011F48E7E886194FD877E08950C944C0E06
:1023B0000E942E138FE39CE90197F1F700C0000003
:1023C0000E942E1380E00E94121280FF04C00E941F
:1023D000D6110C946B1808950C94D8110E94520ECB
:1023E000811102C00E94FA0E0E945D0E8093480285
:1023F0000E94650E90938102809380020E94EC11EE
:102400000E94610E682F70E080E090E00E945A0800
:102410006091B4017091B5018091B6019091B701BE
:102420000C949208E82FF0E0EE0FFF1FE657FD4FE7
:10243000808191810895CF92DF92EF92FF920F9366
:102440001F93CF93DF9382E991E00E940D028AE807
:10245000E82E82E0F82EC0E0D0E09DE8C92E91E0A1
:10246000D92E04E811E0DF93CF93DF92CF920E9440
:10247000A6028AE891E00E940D02F70181919191F4
:102480007F010E94A0039F938F931F930F930E943D
:10249000A60282E891E00E940D0221968DB79EB7B8
:1024A00008960FB6F8949EBF0FBE8DBFC430D105FD
:1024B000D1F6DF91CF911F910F91FF90EF90DF90B8
:1024C000CF90089580EA8A95F1F7089500C00895A5
:1024D0000C94621208950C946A120C946B120C9472
:1024E0006A120C946F12F894E82FE295EF70F0E006
:1024F00031A1282F2F7081E090E001C0880F2A952C
:10250000EAF7982F9095932391A392A1892B82A308
:10251000789408950F931F93CF93DF93CFE7D1E083
:1025200089918F3F11F00E94731281E0C338D80760
:10253000B9F7C3E7D1E00FE711E089918F3F11F0C0
:102540000E9473120C171D07C1F7DF91CF911F91E5
:102550000F910895BF92CF92DF92EF92FF920F9367
:102560001F93CF93DF938C01C62FD0E0CE0181580B
:102570009E4F6C01FC0190819F3F09F450C0B62E24
:10258000F894E92FE295EF70F0E081A19F7021E0CF
:1025900030E001C0220F9A95EAF7822B81A382A135
:1025A0002095282322A378940E946612E3E7F1E0A5
:1025B0004FE751E021E030E0E12CF12C61916F3FD9
:1025C00089F0A62FA295AF70B0E090968C9190E024
:1025D0006F7002C0959587956A95E2F780FD02C0FD
:1025E000C90102C080E090E0E82AF92A220F331FD7
:1025F0004E175F0719F7F60180818F3F11F00E9497
:10260000731261E0E114F10409F460E08B2D0E9483
:102610006812CC0FDD1FC00FD11FF982E882DF9155
:10262000CF911F910F91FF90EF90DF90CF90BF90CF
:1026300008950E948A1288E0EAE8F2E0DF01982F0C
:102640001D929A95E9F7E2E8F2E0DF011D928A9582
:10265000E9F784E00E9479130C940103FF920F9331
:102660001F93CF93DF93CDB7DEB728970FB6F894BB
:10267000DEBF0FBECDBF8E010F5F1F4F88E0F80198
:1026800011928A95E9F7F12C6F2DC8010E94AA12C8
:10269000F394F4E0FF12F8CF48E050E0B80182E88C
:1026A00092E00E942120FF24F394009709F4F12C7A
:1026B000892B41F088E0F801A2E8B2E001900D9288
:1026C0008A95E1F72F2D44E06AE872E082E892E013
:1026D0000E947A130E9403038F2D28960FB6F89458
:1026E000DEBF0FBECDBFDF91CF911F910F91FF9045
:1026F00008950895FF920F931F93CF93DF93F82EC1
:10270000092F162FD72FC42F222349F081E0809361
:102710004B020E941E1890934A02809349028091B6
:102720004B028823D9F08091490290914A020E947D
:102730003618059798F0EF2DF02FA12FBD2F80E0D0
:1027400090E04C2F50E08417950734F4219131919B
:102750002D933D930196F7CF10924B02DF91CF91CD
:102760001F910F91FF9008950E94D51A0E943E0F6D
:102770000C94E11A0E94E51A0E94E10F0C94031BCD
:102780000E94BC170E94BC1A0E942C0F0E94B41316
:102790000E94BA130E94360FFBCFCF93DF93EC0158
:1027A000FB018281882309F43CC1C430FDE5DF07C9
:1027B00060F4CB3F9CE5D90788F49E0122503C454C
:1027C0002431310508F02EC109C0C236EDE5DE071F
:1027D00029F0C63AFDE5DF0709F024C10E94650E25
:1027E0009093810280938002C1318CE5D80709F46F
:1027F000C6C008F042C0C930ECE5DE0709F49BC052
:1028000000F5C5308CE5D80709F485C078F4C330ED
:10281000ECE5DE0709F478C008F07AC0C230DC4588
:1028200009F0F5C0809180028160EFC0C7309CE55F
:10283000D90709F478C008F07AC0809180028061DD
:10284000E4C0CD30FCE5DF0709F487C058F4CB3095
:102850009CE5D90709F479C008F07BC0809180021B
:1028600088606FC0CF30FCE5DF0709F480C008F056
:1028700082C080918002877FC8C0CE3F9CE5D90787
:1028800009F471C000F5C531FCE5DF0709F485C026
:1028900068F4C3319CE5D90709F475C008F095C008
:1028A0000E940208809180028F77AFC0CC3FFCE588
:1028B000DF07A9F108F054C0CB3FDC4509F0A7C001
:1028C0008091810240C0C230EDE5DE0709F489C085
:1028D00058F4C1158DE5D80709F45AC008F069C04D
:1028E0008091810282602FC0C236EDE5DE0709F4D7
:1028F0007CC0C63AFDE5DF0709F481C0C330DD4581
:1029000009F085C080E06EC08091800282607DC049
:102910008091800216C080918002886076C080918C
:10292000810282604FC08091800280626EC080917F
:10293000800280646AC00E940208809180028068E0
:1029400064C0846062C081603DC0809180028E7FDF
:102950005CC0809180028D7F58C08091800216C03B
:102960008091810218C0809181028D7F2BC080915F
:1029700080028F7E4AC0809180028F7D46C0809108
:1029800080028F7B42C080918002877F8B7F3DC019
:10299000809181028D7F8E7F15C08091800282FBA5
:1029A000222720F991E0922790FB82F990FB83F98E
:1029B0002CC080918102982F909591708E7F892BE9
:1029C00090FB81F98093810222C00E9402088091CD
:1029D000800287FB222720F991E0922790FB87F95C
:1029E00014C081E00E94FC0E12C08091800284FB22
:1029F000222720F991E0922790FB84F906C080916C
:102A00008002982F909590FB80F9809380028091AE
:102A10008002909181020E94760E0E94020880E05E
:102A200001C081E0DF91CF910895CF93DF9386318C
:102A30009C4541F5EB010E94550D982F8A8120910C
:102A4000020130910301882379F09A7A81E009F438
:102A500080E080934C02911102C069E201C065E3FD
:102A6000C9010E945A170AC080914C02811102C00C
:102A700069E201C065E3C9010E9465170E94970DD4
:102A800080E001C081E0DF91CF9108950F931F9303
:102A9000CF93DF93C42FD22FFC0182818823C9F00A
:102AA00040934F020E941E1890934E0280934D0255
:102AB00080E28C0F883008F057C0C77081E001C0F9
:102AC000880FCA95EAF7DF91CF911F910F910C946F
:102AD0006E0580914F02481330C080914D02909155
:102AE0004E020E943618883C910538F510E21D0F01
:102AF000CD17B9F080E28C0F883040F4C77081E0C8
:102B000001C0880FCA95EAF70E947505183028F5AC
:102B100081E09D2F977001C0880F9A95EAF70E9477
:102B20006E05802F0E9465051830F0F4D77081E0A3
:102B300001C0880FDA95EAF70AC080E28C0F88306E
:102B400098F4C77081E001C0880FCA95EAF7DF9159
:102B5000CF911F910F910C947505802FDF91CF912C
:102B60001F910F910C946505DF91CF911F910F91EB
:102B700008950F939C01CB01243F4CE5340731F1BC
:102B800088F4293DFCE53F07D9F02A3D4CE53407A0
:102B900079F1283D3C45A9F506E221EE41EE68EDCC
:102BA0007CE52BC0263FFCE53F07E1F0A8F0273F7E
:102BB0003C4539F507E225EE46EE67EF7CE51DC0A2
:102BC00007E225EE45EE69ED7CE517C006E221EE51
:102BD00040EE64EF7CE511C007E225EE44EE65EFC0
:102BE0007CE50BC006E221EE42EE66EF7CE505C017
:102BF00008E221E045EE6AED7CE50E94461580E0A2
:102C000008C0FC018281882319F010924F0201C094
:102C100081E00F910895909393018093920108951C
:102C200090935502809354020895E0915402F091DC
:102C30005502309721F00190F081E02D099480E059
:102C40000895EF92FF921F93CF93DF93FC01A09121
:102C50005402B0915502109709F442C080911001BE
:102C6000882341F08091800287FF04C080818183A6
:102C700086E08083EF011296ED91FC911397CE01CF
:102C800009958091480282FF2BC080FF04C081EB30
:102C900091E00E940D0218E08BEAE82E81E0F82E08
:102CA0008091480280FF0BC088811F928F93FF9212
:102CB000EF920E94A6020F900F900F900F9011506C
:102CC00021961111EDCF8091480280FF09C089EA59
:102CD00091E0DF91CF911F91FF90EF900C940D0246
:102CE000DF91CF911F91FF90EF90089520915202B4
:102CF000309153022817390771F090935302809353
:102D00005202E0915402F0915502309721F0068072
:102D1000F781E02D099408952091500230915102DD
:102D20002817390771F09093510280935002E09177
:102D30005402F0915502309721F00084F185E02D86
:102D400009940895FC01329680911001882331F096
:102D50008091800287FF02C09EE101C096E080E082
:102D6000915028F021912223D9F38F5FF9CF089554
:102D7000662351F1209110012223E9F02091800275
:102D800027FF19C0462F4695469546954E31E0F4EB
:102D9000677021E030E002C0220F331F6A95E2F72E
:102DA000FC01E40FF11D828190E02823392381E0AA
:102DB000232B69F409C0FC01329608962191621711
:102DC00029F0E817F907D1F780E0089581E0089528
:102DD0009C01FC0132969FEF80E04191461789F0FB
:102DE0009F3F19F4411101C0982F8F5F8630A9F7DA
:102DF0009F3F39F0F901E90FF11D97FDFA956283C4
:102E0000089508959C012A5F3F4FFC0142814613BB
:102E100001C01282019682179307B9F70895262FF1
:102E20002695269526952E3170F4FC01E20FF11DB2
:102E3000677021E030E001C0220F6A95EAF78281D5
:102E4000282B228308958091480280FF0CC01F9296
:102E50006F9381EE91E09F938F930E94A6020F9053
:102E60000F900F900F900895262F26952695269562
:102E70002E3178F4FC01E20FF11D677021E030E0A3
:102E800001C0220F6A95EAF72095828128232283C8
:102E900008958091480280FF0CC01F926F9383ECCD
:102EA00091E09F938F930E94A6020F900F900F9036
:102EB0000F90089520911001222329F02091800283
:102EC00027FD0C940F170C94E81620911001222373
:102ED00029F02091800227FD0C9434170C940217DE
:102EE00020911001FC013296222331F08091800262
:102EF00087FF02C08EE101C086E0DF011D928A9546
:102F0000E9F7089508950C94821783E080935602A0
:102F10000C948317811102C081E001C082E080938C
:102F200056020C9483170C948A1781E08093560202
:102F30000C9483170C94951708950C949C170C947B
:102F40009D170C949C170C949C170C949C17CF9372
:102F50000E94A3170E942E130E94A117C0E08C2F7D
:102F60000E941212892B29F4CF5FC430C1F780E090
:102F700001C081E0CF91089508951F920F920FB67E
:102F80000F9211248F939F93AF93BF938091570219
:102F9000811113C08091920290919302A0919402AA
:102FA000B09195024196A11DB11D8093920290931C
:102FB0009302A0939402B0939502BF91AF919F9119
:102FC0008F910F900FBE0F901F90189580919A02CD
:102FD000843031F10E9486031092570220E488E188
:102FE00090E00FB6F894A895809360000FBE2093F0
:102FF000600083B7817F846083BF83B7816083BFB4
:103000007894889583B78E7F83BF0FB6F894A89580
:1030100080916000886180936000109260000FBE14
:1030200008950E9402080C948A0382E084BD93E014
:1030300095BD9AEF97BD80936E0008952FB7F894D1
:103040008091920290919302A0919402B091950286
:103050002FBF08952FB7F894609192027091930258
:1030600080919402909195022FBF08959C014FB7D3
:10307000F8948091920290919302A0919402B09161
:1030800095024FBF821B930B089578941F920F9265
:103090000FB60F9211248F939F93AF93BF9380919C
:1030A000920290919302A0919402B09195020196A0
:1030B000A11DB11D8093920290939302A09394025C
:1030C000B0939502BF91AF919F918F910F900FBEDA
:1030D0000F901F90189581E08093E00080E280932C
:1030E000D8001092C9008FE19EE40197F1F700C06B
:1030F000000087E090EBDC018093A3029093A40290
:10310000A093A502B093A6029CE088E10FB6F894C4
:10311000A895809360000FBE90936000FFCF8091D0
:103120007E0208950895CF93DF932091100122230A
:1031300039F02091800227FF03C060E222E002C044
:1031400068E021E02093E9002FEF3091E800215062
:1031500035FD06C035ED3A95F1F700002111F5CFA8
:103160002091E80025FF1DC0EC0180911001811124
:1031700005C040E050E068E070E003C070E040E06F
:1031800050E0CE010E94721B8091E8008E77809300
:10319000E80080E2FE01AEE5B2E001900D928A9572
:1031A000E1F7DF91CF91089580935A0270935C020A
:1031B00060935B0280919A02843001F582E08093F3
:1031C000E9008FEF9091E800815095FD06C095EDE4
:1031D0009A95F1F700008111F5CF8091E80085FF05
:1031E0000DC040E050E063E070E08AE592E00E94AC
:1031F000721B8091E8008E778093E8000895BC01EF
:1032000084E00C94D418BC0183E00C94D418089585
:1032100083E192E00E940D0280919902811109C020
:103220000E94031D0E94601D8091E20084608093D3
:10323000E20008958FE092E00E940D021092990240
:1032400008958BE092E00E940D020C949A1787E09B
:1032500092E00E940D026091960281E0611101C02E
:1032600080E00C94851783E092E00E940D0290911B
:103270009A0281E0943009F080E0609196020C940B
:103280008A17209159022F5F822F62E30E940F203C
:10329000992319F0209359020895109259028091B0
:1032A0005D02882371F180919A02843041F580910A
:1032B000E9008F702091EC00922F917020FD90E832
:1032C000892B93E09093E9009091EB0090FF14C05C
:1032D0009091EE0097FF10C09091E80095FF03C019
:1032E0001092F100F9CF9091E80090FF05C0909105
:1032F000E8009E779093E8008F708093E900109229
:103300005D02089542E061EC81E00E947C1C42E293
:1033100061EC82E00E947C1C42E261EC83E00E944E
:103320007C1C90919A0281E0943009F080E06091D9
:1033300096020C94931780919C02833009F461C02B
:1033400030F4813071F0823009F49AC008958A30E7
:1033500009F486C08B3009F46CC0893009F0A8C02C
:1033600020C080919B02813A09F0A2C08091E800C0
:10337000877F8093E80080919F029091A002892B23
:1033800021F460E28EE592E003C060E080E090E02E
:1033900070E00E94BD1B8091E8008B778093E8006D
:1033A000089580919B02813209F082C080919F0232
:1033B0009091A002029708F07BC08091E800877F7F
:1033C0008093E8008091E80082FD05C080919A0218
:1033D0008111F8CF6DC02091F3008091F20090E050
:1033E000922B029731F48091F100813011F08630F8
:1033F00021F48091F10080937E028091E8008B7728
:1034000053C080919B02813A09F052C080919F0283
:103410009091A002892B09F04BC08091E800877F32
:103420008093E8008091E80080FFFCCF809110013C
:1034300036C080919B028132D9F580919F02909194
:10344000A002892BA9F58091E800877F8093E8008E
:103450000E94B11C80919D02809310010C9402087F
:1034600080919B02813221F58091E800877F8093D3
:10347000E8000E94B11C80919E0280937F02089513
:1034800080919B02813AA1F48091E800877F80932C
:10349000E8008091E80080FFFCCF80917F0280935C
:1034A000F1008091E8008E778093E8000C94B11CC5
:1034B00008959FB7F89410925D029FBF90919A0271
:1034C000943009F057C09091E9009F703091EC0062
:1034D000232F217030FD20E8922B23E02093E90078
:1034E0002091EB0020FF43C02091EE0027FF3FC05A
:1034F00020915802222321F02091E80025FF37C0B7
:103500001092580226E03091E80035FD15C0309148
:103510009A02343061F53091EB0035FD28C021501E
:1035200021F481E08093580222C0EFE9FFE0319757
:10353000F1F700C00000E7CF8093F1008091E80030
:1035400085FD0AC08091E80080FFFCCF8091E800F3
:103550008E778093E80006C08FB7F89421E020931F
:103560005D028FBF9F709093E90080E008959F7087
:103570009093E9008FEF089584B7877F84BF0FB6DB
:10358000F894A89580916000886180936000109203
:1035900060000FBE90E080E80FB6F8948093610061
:1035A000909361000FBE0C9495170E94031D0E941A
:1035B000601DE2EEF0E080818460808378940C945A
:1035C000F41F84E091E00C94101680919A028530EB
:1035D000C9F48FEF91E00E940D0280919A0285302C
:1035E00079F40E94E617809198028823B1F30E9433
:1035F000A717882391F30E945C1B0E940208EDCF5D
:103600000C941118089508950C94061B292F332744
:1036100023303105C9F060F42130310581F02230CA
:10362000310509F041C08BE590E021E532E040C072
:1036300021323105E1F02232310531F135C082E12C
:1036400090E02CEA32E034C099278130910549F0AE
:1036500028F0029749F5E7E1F2E005C0EDE4F2E079
:1036600002C0E9E2F2E0849190E09F0121C0633062
:103670007105D0F4660F771FFB01E457FE4F2081E0
:10368000318189E090E014C06330710568F4FB017A
:10369000EE0FFF1FEA57FE4F20813181FB01ED57EE
:1036A000FE4F808190E004C080E090E020E030E0B8
:1036B000FA0131832083089580E189BD82E189BDCB
:1036C00009B400FEFDCF8091D8008F7D8093D80093
:1036D0008091E00082608093E0008091E00081FDB5
:1036E000FCCF0895CF92DF92EF92FF920F931F933A
:1036F000CF93DF93EC018B017A010E94D01C8111E2
:1037000033C0E114F10439F0F70180819181081B85
:10371000190BC80FD91FC12CD12C0115110519F196
:103720008091E80085FD16C08091E8008E77809337
:10373000E800E114F10449F0F70180819181C80E9D
:10374000D91ED182C08285E00FC00E94D01C882380
:1037500021F30AC089918093F10001501109FFEF14
:10376000CF1ADF0ADACF80E0DF91CF911F910F915E
:10377000FF90EF90DF90CF9008952091A1023091BB
:10378000A2022617370748F06115710539F4209118
:10379000E8002E772093E80001C0B901FC0120E089
:1037A0006115710579F180919A028823F1F18530D4
:1037B000F1F18091E80083FD3CC08091E80082FD3A
:1037C0002EC08091E80080FFEBCF2091F300809124
:1037D000F20090E0922B6115710551F0883091054F
:1037E00038F421912093F100615071090196F3CFD3
:1037F00021E0089709F020E08091E8008E7780931F
:10380000E800CECF2111CFCF0AC080919A02882341
:1038100061F0853061F08091E80083FD0AC08091FD
:10382000E80082FFF2CF80E0089582E0089583E00F
:10383000089581E008952091A1023091A2022617F7
:10384000370748F06115710539F42091E8002E77AB
:103850002093E80001C0B901FC0120E06115710569
:1038600091F180919A02882309F440C0853009F4CF
:103870003FC08091E80083FD3DC08091E80082FD5B
:103880002FC08091E80080FFE9CF2091F300809164
:10389000F20090E0922B6115710559F08830910586
:1038A00040F424912093F100319661507109019602
:1038B000F2CF21E0089709F020E08091E8008E77B0
:1038C0008093E800CBCF2111CCCF0AC080919A021F
:1038D000882361F0853061F08091E80083FD0AC0A3
:1038E0008091E80082FFF2CF80E0089582E00895A1
:1038F00083E0089581E00895982F973068F59093BC
:10390000E900981739F07091EC002091ED0050918A
:10391000F00003C0242F762F50E021FD02C09F5FEE
:10392000ECCF3091EB003E7F3093EB003091ED0017
:103930003D7F3093ED003091EB0031603093EB0030
:103940007093EC002093ED005093F0002091EE0076
:1039500027FDE5CF80E008958F708093E90081E036
:10396000089580919B0287FF11C08091E80082FD3D
:1039700005C080919A028111F8CF11C08091E800B2
:103980008B770BC080919A02882349F08091E800E0
:1039900080FFF8CF8091E8008E778093E80008954B
:1039A0002091E4003091E50095E64091EC00842FF1
:1039B000817040FF23C08091E80080FD1DC0809190
:1039C0009A02882399F0853099F08091EB0085FD6B
:1039D00011C04091E4005091E5002417350729F308
:1039E000915011F09A01E1CF84E0089582E00895AA
:1039F00083E0089581E0089580E008954091E80013
:103A000042FFDDCF08950E94711D0E94791DE0EEF6
:103A1000F0E0808181608083E8EDF0E080818F7745
:103A2000808319BCA7EDB0E08C918E7F8C93808150
:103A30008F7E80831092990208950F931F93CF93E6
:103A4000DF930E94711D0E94791DC8EDD0E088812E
:103A50008F77888388818068888388818F7D888339
:103A600019BC10929A02109296021092980210922B
:103A7000970200EE10E0F80180818B7F80838881BF
:103A80008160888342E060E080E00E947C1CE1EE7F
:103A9000F0E080818E7F8083E2EEF0E080818160C3
:103AA0008083808188608083F80180818E7F80831D
:103AB000888180618883DF91CF911F910F91089554
:103AC000E8EDF0E080818F7E8083E7EDF0E080819B
:103AD0008160808384E082BF81E0809399020C94AE
:103AE0001D1DE8EDF0E080818E7F80831092E20062
:103AF00008951092DA001092E10008951F920F923B
:103B00000FB60F9211242F933F934F935F936F93B0
:103B10007F938F939F93AF93BF93EF93FF93809186
:103B2000E10082FF0BC08091E20082FF07C080911C
:103B3000E1008B7F8093E1000E9441198091DA00BF
:103B400080FF1FC08091D80080FF1BC08091DA00E9
:103B50008E7F8093DA008091D90080FF0DC080E1D4
:103B600089BD82E189BD09B400FEFDCF81E080936B
:103B70009A020E94081905C019BC10929A020E946C
:103B80001A198091E10080FF19C08091E20080FF46
:103B900015C08091E2008E7F8093E2008091E20068
:103BA00080618093E2008091D80080628093D80089
:103BB00019BC85E080939A020E9427198091E10048
:103BC00084FF30C08091E20084FF2CC080E189BD79
:103BD00082E189BD09B400FEFDCF8091D8008F7DC0
:103BE0008093D8008091E1008F7E8093E1008091E6
:103BF000E2008F7E8093E2008091E20081608093FA
:103C0000E20080919602882311F084E007C0809141
:103C1000E30087FD02C081E001C083E080939A0247
:103C20000E9433198091E10083FF29C08091E20056
:103C300083FF25C08091E100877F8093E10082E0CF
:103C400080939A02109296028091E1008E7F809379
:103C5000E1008091E2008E7F8093E2008091E2009B
:103C600080618093E20042E060E080E00E947C1C82
:103C70008091F00088608093F0000E942119FF91EC
:103C8000EF91BF91AF919F918F917F916F915F91D4
:103C90004F913F912F910F900FBE0F901F9018954D
:103CA0001F920F920FB60F9211242F933F934F93B1
:103CB0005F936F937F938F939F93AF93BF93CF93B4
:103CC000DF93EF93FF93C091E900CF708091EC00F8
:103CD000D82FD17080FDD0E81092E9008091F000DB
:103CE000877F8093F00078940E94941E1092E900E0
:103CF0008091F00088608093F000CD2BCF70C0934E
:103D0000E900FF91EF91DF91CF91BF91AF919F912A
:103D10008F917F916F915F914F913F912F910F9074
:103D20000FBE0F901F9018951F93CF93DF93CDB7C1
:103D3000DEB7AA970FB6F894DEBF0FBECDBFEBE992
:103D4000F2E08091F100819322E0E33AF207C9F7B3
:103D50000E949B198091E80083FF2EC180919B02F5
:103D600090919C02492F50E04A30510508F024C13F
:103D7000FA01EE59FF4F0C941B20803821F0823855
:103D800009F01AC108C08091970290919802992376
:103D900089F082600FC080919F028F70873008F099
:103DA0000BC18093E9008091EB0085FB882780F9A7
:103DB0001092E9009091E800977F9093E80080933B
:103DC000F1001092F100D1C0282F2D7F09F0F4C02E
:103DD000882319F0823061F0EFC080919D0281301C
:103DE00009F0EAC0933009F080E0809398022EC079
:103DF00080919D0281112AC080919F028F702FEFC8
:103E0000280F263008F0D8C08093E9002091EB00FD
:103E100020FF1CC0933021F48091EB00806214C01D
:103E20009091EB0090619093EB0021E030E0A901CC
:103E300002C0440F551F8A95E2F74093EA001092A2
:103E4000EA008091EB0088608093EB001092E9001B
:103E50008091E800877F8093E8000E94B11CACC08D
:103E60008111AAC010919D021F778091E300807894
:103E7000812B8093E3008091E800877F8093E800A6
:103E80000E94B11C8091E80080FFFCCF8091E3008C
:103E900080688093E300111102C082E001C083E0DA
:103EA00080939A0289C08058823008F085C0809142
:103EB0009D0290919E028C3D53E0950779F583E039
:103EC0008A838AE289834FB7F894DE01139620E053
:103ED0003EE051E2E32FF0E050935700E49120FFE1
:103EE00003C0E295EF703F5FEF708E2F90E0EA30F5
:103EF00010F0C79601C0C0968D939D932F5F24311B
:103F000049F74FBF8091E800877F8093E8006AE21D
:103F100070E0CE0101960E94BD1B16C060919F0209
:103F20007091A002AE014F5F5F4F0E94041BBC0165
:103F3000892B09F441C09091E800977F9093E800A5
:103F400089819A810E941B1C8091E8008B77809365
:103F5000E80032C0803881F58091E800877F809347
:103F6000E800809196028093F1008091E8008E77BE
:103F700072CF811121C080919D0290919E0299275C
:103F80000297D4F48091E800877F8093E8008091C5
:103F90009D02809396020E94B11C8091960281112D
:103FA00006C08091E30087FD02C081E001C084E08B
:103FB00080939A020E9482198091E80083FF0AC0D0
:103FC0008091E800877F8093E8008091EB00806219
:103FD0008093EB00AA960FB6F894DEBF0FBECDBF5C
:103FE000DF91CF911F910895CF9380919A028823FA
:103FF000A1F0C091E900CF709091EC00892F817001
:1040000090FD80E8C82B1092E9008091E80083FDC4
:104010000E94941ECF70C093E900CF910895991B20
:1040200079E004C0991F961708F0961B881F7A95AF
:10403000C9F780950895EE0FFF1F0590F491E02DCC
:104040000994FB01DC0104C08D910190801921F4D9
:1040500041505040C8F7881B990B0895F999FECF3D
:1040600092BD81BDF89A992780B50895A8E1B0E086
:1040700042E050E00C946220262FF999FECF92BDC9
:1040800081BDF89A019700B4021639F01FBA20BD1D
:104090000FB6F894FA9AF99A0FBE08950396272F4F
:1040A0000E943D200E943C20252F0E943D20242F6D
:1040B0000C943D200196272F0E943D200C943C201B
:1040C000DC01CB01FC01F999FECF06C0F2BDE1BDD8
:1040D000F89A319600B40D9241505040B8F70895C7
:0440E000F894FFCF82
:1040E400C80016028F18931807190319FF1892189D
:1040F40001E200E900EA00B500B600B700CD008394
:1041040001CC008A01920194012102230224022598
:1041140002260227022A02B300B4006F0070008155
:104124008283E200E900EA00B500B600B700CD00E2
:104134008301CC008A01920194012102230224020A
:104144002502260227022A02B300B4006F00700081
:10415400818283F1F4F53435363792939594963011
:10416400313233406D224D03E002BE0263027C0211
:024174009502B2
:00000001FF
